:020000040000FA
:0200000075D1B8
:0200080047D0DF
:080018000B6ED8CF0AF0F29440
:100020000F0E89129212EC0E8A1293120C50F926BE
:1000300020D00FD089960F0E0D140809921AE00EE9
:100040000D14931A0DB69396938410B693940C6A7C
:100050001FD089940F0E0E140409921AE00E0E148C
:10006000931A0EB4939693842DA29394040E0C6E5F
:100070000FD089900F0E0F140109921AE00E0F1481
:10008000931A0FB09396938410B29394020E0C6E51
:100090000B500AC0D8FF10009E921B661B062266FA
:1000A00022061D2E0FD0640E1D6E202A1E2E04D097
:1000B0003C0E1E6E1C661C061F2E04D03C0E1F6ECE
:1000C0001AAE212A172E1100020E176E1850500B6F
:0E00D000196E8050500B186E1962188E1100B8
:100200006F6F6F066FAB6F8F6FC66FCD6FED6F0740
:100210006FEF6FCF066F060606AB068F06C606CDDC
:1002200006ED060706EF06CFAB6FAB06ABABAB8FA9
:10023000ABC6ABCDABEDAB07ABEFABCF8F6F8F06E4
:100240008FAB8F8F8FC68FCD8FED8F078FEF8FCFB7
:10025000C66FC606C6ABC68FC6C6C6CDC6EDC60738
:10026000C6EFC6CFCD6FCD06CDABCD8FCDC6CDCD34
:10027000CDEDCD07CDEFCDCFED6FED06EDABED8F35
:10028000EDC6EDCDEDEDED07EDEFEDCF076F070618
:1002900007AB078F07C607CD07ED070707EF07CFA7
:1002A000EF6FEF06EFABEF8FEFC6EFCDEFEDEF07A0
:1002B000EFEFEFCFCF6FCF06CFABCF8FCFC6CFCD86
:1002C000CFEDCF07CFEFCFCF00010102020304042F
:1002D00005060607080809090000000200040005D9
:1002E000000700090101010301040106D350700950
:1002F000D36E896A7F0EC16E500E926E8A6A030EAB
:10030000936E09EC02F01DEC02F00850AA0A0AE014
:1003100009EC02F0230E046E0A0E056E010E026E49
:10032000140E066E500E186E050E176E050E426EF8
:100330002C6A3C0E1F6E1E6E640E1D6EC30ED56EB3
:10034000D66ACA6ACC6A2B0ECA6ED00ECB6ECA842D
:10035000F26A9D6AA06A9E6AC00EF06EC10EF16ECE
:10036000020E9F6ED08E9D82E00EF26EEF0E0F6E2B
:10037000EF0E0E6EEF0E0D6E10861082898E8A883B
:10038000FA0E05EC02F0899E8A98106ACCEC02F015
:10039000FDE14CEC02F0CC0EABEC02F0440EABEC09
:1003A00002F02C0E0F6E6F0E0E6EED0E0D6EC80E5F
:1003B00005EC02F0DDEC06F0D18018A807EC05F0A2
:1003C00018AC2DEC07F0040073EC03F0C0EC04F063
:1003D000E4EC04F0EDEC04F0F0D7116E112611C03E
:1003E000F6FF020EF76E0900F5CF11F00800F5CF09
:1003F00012F01200189E1B6E189018AE03D0189EB3
:10040000188012001B66F9D712001B6E1B66FED700
:10041000120000EE00F0EE6AEAA0FDD71200AA0E6C
:10042000086E446A090E456E00EE00F0EE502AECAC
:1004300002F0442A452EFAD71200446A090E456E8E
:1004400000EE00F044503BEC02F0EE6E442A452EE4
:10045000F9D71200A6B2FED7A86E44C0A9FFA69E87
:10046000A69CA684F29E550EA76EAA0EA76EA68223
:10047000F28EA6941200A96EA69EA69CA680A850F5
:10048000120000000000000000000000000000005A
:10049000262EF7D700001200190E276E000000006C
:1004A0009380010E266E000000000000000041EC69
:1004B00002F08A909390770E266E000000000000F4
:1004C000000041EC02F0F29E93800D0E266E0000BB
:1004D00000000000000041EC02F08150010B272ECB
:1004E000FCE1286EF28E4F0E266E00000000000028
:1004F000000041EC02F01200080E256EF29E8A9078
:1005000093900000000000000000000000000000C8
:1005100000000000938000000000000000000000C8
:1005200000000000000000000000000000000000CB
:10053000000000008150010BFF0F2932090E266ECA
:10054000000000000000000041EC02F0F28E252EB9
:10055000D5D729501200296E080E256EF29E8A907A
:100560009390010E266E000000000000000041EC98
:1005700002F02932D8B093800B0E266E00000000E6
:100580000000000041EC02F0938000000000000039
:10059000F28E252EE3D712000000938000000000A9
:1005A000000000000000000081A023D04CEC02F00D
:1005B0004CEC02F028500EE1330EABEC02F07CEC78
:1005C00002F02C6E100E2C1804E0280E2C1801E0FE
:1005D000AED1000C190E276E9380010E266E00001E
:1005E00000000000000041EC02F081B01BD0272E7B
:1005F000F3D7F28E2D828A98898EE10E0F6E680EE7
:100600000E6EE00E0D6EC80E05EC02F0DDEC06F08D
:10061000680E0E6EAC0E0D6EC80E05EC02F02C6668
:100620001200FF008A909390770E266E0000000063
:100630000000000041EC02F0F29E9380190E436E20
:100640000D0E266E000000000000000041EC02F0DC
:1006500081A01BD0432EFCD7F28E2D828A98898EE2
:10066000E10E0F6E680E0E6EE00E0D6EC80E05ECFC
:1006700002F0670E0F6EAC0E0E6EE00E0D6EC80E21
:1006800005EC02F02C661200FF00F28E2D828A9893
:10069000898EE10E0F6E680E0E6EE00E0D6EC80EA6
:1006A00005EC02F0A00E0F6EE90E0E6ECD0E0D6E73
:1006B000C80E05EC02F02C661200FF00F28E2D82AF
:1006C000690E0F6EA00E0E6E690E0D6EC80E05EC53
:1006D00002F0E90E0F6EA00E0E6EA00E0D6EC80E8B
:1006E00005EC02F012007CEC02F0010F24E00A0E8F
:1006F00005EC02F0362A140E36621200366AF28ECB
:100700002D82A00E0F6EAE0E0E6E0D6AC80E05EC99
:1007100002F04CEC02F0CC0EABEC02F0440EABEC71
:1007200002F0E90E0F6EA00E0E6EA00E0D6EC80E3A
:1007300005EC02F01200366A4CEC02F028664AD74B
:10074000CC0EABEC02F0BE0EABEC02F07CEC02F097
:100750002A6E336A346AADEC04F07CEC02F02B6E46
:10076000ADEC04F07CEC02F0ADEC04F07CEC02F0BB
:10077000ADEC04F07CEC02F0ADEC04F07CEC02F0AB
:10078000ADEC04F07CEC02F02F6EADEC04F07CECF0
:1007900002F02E6EADEC04F07CEC02F0ADEC04F057
:1007A00033508CE134A08AE04CEC02F0CC0EABEC80
:1007B00002F0440EABEC02F04266424E02D01A84C4
:1007C00009D02A503C5C2B50D8A0010F3D5C800B17
:1007D000D8A406D02AC03CF02BC03DF02FC040F07A
:1007E0001AB409D02A503E5C2B50D8A0010F3F5CB0
:1007F000800BD8B407D02AC03EF02BC03FF02FC0EA
:1008000041F01A942D6A2B50F00BF00AD8B42D80C9
:10081000100E2C1804E0280E2C1825E088D0D89053
:100820002A30306E100E2E180AE02AB005D0316A38
:100830002DA024D0300622D0050E316E1FD02F50AF
:100840002E5E2DA006D02E5002E1300602D01008F8
:100850002E6E020EF76E2EC0F6FFC80EF6260800AA
:10086000F550316E0BD00F0E2A142E6E070E2B147E
:10087000306EF00E2A143012303AE3D72DA003D098
:1008800030507F08306E30C03AF031C03BF007A0E6
:1008900006D0E2EC06F038C03AF039C03BF0C70EA3
:1008A0003A640CD0C80E3A5CEDEC01F011C00EF0C9
:1008B00012C00DF0AB0E0F6E2D82000C630E3A6469
:1008C0000CD0640E3A5CEDEC01F011C00EF012C0D9
:1008D0000DF0060E0F6E2D82000C3A50EDEC01F07B
:1008E0007AEC04F02DB2000C3B50EDEC01F012C09C
:1008F0000DF0000C2DA004D007A00BD02DB409D012
:100900006F0E116201D0116A11C00FF012C00EF00B
:100910001200800E0F6E0A0E3A6003D012C00EF065
:10092000120011C00EF012C00DF02D821200F28ED6
:100930002D828A98898E200E0F6EAE0E0E6E0D6A75
:10094000C80E05EC02F0E90E0F6EA00E0E6EA00EA2
:100950000D6EC80E05EC02F0EAD7326E080E356E49
:1009600032503318136E1330335001E3180A136EEC
:100970001330336E01E034803242352EF1D712004D
:1009800000B00BD02DB018D03A50066401D014D06E
:10099000025006243A600AD016D02DB003D03A5047
:1009A00006640AD00250065C3A600DD01C660BD07B
:1009B0008A9801C01CF007D01C6605D01ABE03D06F
:1009C0008A8801C01CF012003A50046404D005600B
:1009D00002D0899E1200898E1200036601D002D0D7
:1009E00081B206D010961A9E3C0E1F6E216A12002C
:1009F0001ABE05D010860350216001D01200226675
:100A000003D01076210E226E1A8E8A9812001A8256
:100A10002D82206A0400020E206064D0DDEC06F016
:100A200018A8F8D70400280E236E030E246E065073
:100A30009BEC06F018AC2EEC05F00F0E18B005EC90
:100A400002F0189018A850EC05F00F0E18B005EC45
:100A500002F01890050E2064E5D760D10400206AEA
:100A600018BC12002350FAEC01F0242E0AD0030E19
:100A7000246E23060A0E236004D00A0E236E18B0DB
:100A80001200062A640E07B0D40E066404D0640E69
:100A900007B0D40E066E06509BEC06F01A80DED727
:100AA0000400206A18B812002350FAEC01F0242E3A
:100AB0000AD0030E246E23060A0E236004D00A0E09
:100AC000236E18B012000606010E07B0200E066055
:100AD00004D0010E07B0200E066E06509BEC06F007
:100AE0001A80DED71A822D82CD0E0F6EE90E0E6EA1
:100AF000E00E0D6E6E0E97EC06F0690E0F6E800E16
:100B00000E6EE60E0D6EC80EFAEC01F0DDEC06F08E
:100B1000E60E00B0690E0D6EC5EC06F018A80CD0FC
:100B200018BCFAD7002A020E0060006AE60E00B078
:100B3000690E0D6E1A80F0D797EC06F0AE0E0F6EB0
:100B4000680E0E6ECE0E0D6EC80EFAEC01F0DDECE6
:100B500006F001509BEC06F0C5EC06F018A80BD08F
:100B600018BCFAD7012A100E0160016A01509BECF3
:100B700006F01A80F1D797EC06F0E60E0F6ECE0E57
:100B80000E6ECD0E0D6EC80EFAEC01F0DDEC06F027
:100B900002509BEC06F0C5EC06F018A80BD018BC70
:100BA000FAD7022A090E0260026A02509BEC06F094
:100BB0001A80F1D797EC06F0AC0E0F6EAE0E0E6EEB
:100BC000AC0E0D6EC80EFAEC01F0DDEC06F0035031
:100BD0009BEC06F0C5EC06F018A80BD018BCFAD7B1
:100BE000032A0B0E0360036A03509BEC06F01A8085
:100BF000F1D797EC06F0E60E0F6E200E0E6EE70EA4
:100C00000D6EC80EFAEC01F0DDEC06F004509BEC22
:100C100006F0C5EC06F0280E236E030E246E18A80D
:100C200022D018BCF6D718BCF6D72350FAEC01F046
:100C3000242E0AD0030E246E23060A0E236004D04D
:100C40000A0E236E18B0E7D7042A640E07B0D40E3C
:100C5000046404D00A0E07B0320E046E04509BECFC
:100C600006F01A80DCD797EC06F0680E0F6EAC0E1B
:100C70000E6EE70E0D6EC80EFAEC01F0DDEC06F01C
:100C800005509BEC06F0C5EC06F0280E236E030E13
:100C9000246E18A822D018BCF6D718BCF6D723505B
:100CA000FAEC01F0242E0AD0030E246E23060A0E5D
:100CB000236004D00A0E236E18B0E7D7052A640E0D
:100CC00007B0D40E056404D0000E07B0200E056EE8
:100CD00005509BEC06F01A80DCD797EC06F0690E05
:100CE0000F6E800E0E6EE10E0D6EC80EFAEC01F066
:100CF000DDEC06F0690E07B0E10E0D6EC5EC06F0F6
:100D000018A80CD018BCFAD7072A020E0760076A89
:100D1000690E07B0E10E0D6E1A80F0D797EC06F061
:100D20001A922D921AB00FEC02F01A9012000400E1
:100D300018A8FDD71200146EC70E14640BD0C80E8D
:100D4000145CEDEC01F011C00EF012C00DF0AB0E12
:100D50000F6E1200630E14640BD0640E145CEDEC85
:100D600001F011C00EF012C00DF0060E0F6E120051
:100D70000F6A1450EDEC01F06F0E116201D0116A90
:100D800011C00EF012C00DF012000FC014F00EC012
:100D900015F00DC016F00F6A0E6A0D6A0A0EFAEC15
:100DA00001F014C00FF015C00EF016C00DF018B011
:100DB0001200140EFAEC01F012000F6A0E6A0D6AAE
:100DC0002D821200090E300217EC07F0F3CF38F035
:100DD000F450F424396E31503124F66E020EF76E61
:100DE000D80EF6260900F55038260800F5503924AB
:100DF0000700376E0F0B396E37380F0B38262DB0C2
:100E000007D02D942D9E200E3826D8B02D8E12009E
:100E100038502008386E04E700082D84386E06D05C
:100E20002D94395003E00A08396E38061200080E76
:100E3000376E050E20EC07F0372EFCD7F336120084
:100E4000F336F436D8A003D0F45ED8801200F45EF6
:100E5000D8B01200F426D8901200206A040E206048
:100E60003BD02D82E60E0F6E200E0E6E0D6A18AC72
:100E7000F5D7640E05EC02F0DDEC06F02D923FC0D4
:100E80002BF03EC02AF041C02FF002EC04F0B40E6B
:100E900005EC02F0DDEC06F0320E05EC02F02D82DE
:100EA000680E0F6EAC0E0E6E0D6A640E05EC02F04D
:100EB000DDEC06F02D923DC02BF03CC02AF040C086
:100EC0002FF002EC04F0B40E05EC02F0DDEC06F0BD
:100ED000320E05EC02F01200020E426E2D82690EF7
:100EE0000F6E680E0E6EA00E0D6EB40E05EC02F0C5
:020EF0001200EE
:020000040030CA
:03000100080A1CCE
:020005008081F8
:0600080003C003E0034009
:00000001FF
